:200000000FC2D4C527C282C325C224C223C222C221C220C21FC21EC21DC21CC21BC21AC2B6
:2000200019C218C217C2040309044203530070006100630065006D0061006E00200053003E
:200040007000690066006600200068007400740070003A002F002F00730079006D006C00BE
:2000600069006E006B002E0064006B001A0353007000690066006600430068006F007200A0
:200080006400650072001201100100000008401CA3059800010200010902220001010080AA
:2000A00032090400000103010100092101010001223F0007058103080014272727002727FE
:2000C00000B4B45000A6A75000BA00BE00C100C50000001A001C001800150000000B001649
:2000E000000C0005000E001D0007000000080017006F00710029003300360000003700678E
:2001000000000049000000650042003D00340070002C0009000A001900060030001300115C
:20012000000F001B000D00140010002F0004001200730000000000000000000000000000AC
:200140000000000000000000000000000000005300660028004F0051002A0046004C004E14
:200160000050004D002B004A00520047004B00390048000000000000000000000000000008
:200180000000000000000000000000000000000000570058005E005A005D00550063005B88
:2001A000005C00590056005F0060005400610062006D0000000000000000000000000000F1
:2001C000000000000000000000000000000000000000002200210076002000000075002DA4
:2001E000001F00310021023500380000002E0074002C007100290033003600000037006BAC
:200200000000004900000069000000000034006D001E002600250030002400300022022F4B
:2002200000230024027700380225022F002E022700730000000000000000000000000000A4
:2002400000000000000000000000000000000053006A0028004F0051002A0046004C004E0F
:200260000050004D002B004A00520047004B00390048000000000000000000000000000007
:200280000000000000000000000000000000000000570058005E005A005D00550063005B87
:2002A000005C00590056005F0060005400610062006D0000000000000000000000000000F0
:2002C000000000000000000000000000000000000000003E003D0000003C00000000000067
:2002E000003B00000000000000000000000000000000006D000000000000000000000067EF
:2003000000000000000000650000000000000000003A0042004100450040000000440000F2
:20032000003F000000000000004300000000000000730000000000000000000000000000C8
:20034000000000000000000000000000000000000066000000000000000000000000000037
:2003600000000000000000000000000000000000000000000000000000000000000000007D
:2003800000000000000000000000000000000000000000000000000000000000000000005D
:2003A00000000000000000000000000000000000006D0000000000000000000000000000D0
:2003C0000000000000000000000000000000000000010204081020408005010906A1010562
:2003E0000719E029E71500250175019508810295017508810395057501050819012905918F
:200400000295017503910395067508150025650507190029658100C0D100D101D102000017
:2004200011241FBECFE5D4E0DEBFCDBF10E0A0E6B0E0E8E2F7E102C005900D92AE36B107DF
:20044000D9F710E0AEE6B0E001C01D92AB3BB107E1F737C3D5CD85B7836085BF8BB78064AD
:200460008BBF83EC8093910008950F931F93CF93DF936091A10016160CF0C8C06350809154
:200480009E00C1EBD0E0C81BD10980919D008D3209F09FC08AE580936100683009F0AEC0FE
:2004A0008881807609F082C02FE830E010928F008981882341F4109290003093A000209378
:2004C0009F0092E07DC0853021F48A818093A200F1C0863009F04CC08B81813041F486E878
:2004E00090E09093A00080939F0092E1E6C0823041F488E990E09093A00080939F0092E24D
:20050000DCC0833001F58A81882341F486E290E09093A00080939F0094E0CFC0813041F475
:200520008AE290E09093A00080939F0092E4C5C0823009F0C1C08CE690E09093A00080938B
:200540009F009AE1BAC0813241F48AEA90E09093A00080939F0099E0B0C0823209F0ACC0C4
:2005600089ED93E09093A00080939F009FE3A5C0883039F484EA90E09093A00080939F00FE
:200580000CC0893021F48A818093A40093C08A3031F43093A00020939F0091E011C08B301B
:2005A00009F088C083EC8093910084C0CE01C3D0982F8F3F29F4888187FF1CC09E811AC02B
:2005C00020E88F818823E1F48E818917C8F4982F17C080916E0087FD11C0CE01ECD08F3F4D
:2005E00031F4809360008EE18093610005C0882319F090E020E004C09FEFFCCF90E020E802
:2006000020936E00909360001092A1008091610084FF45C0809160008F3F09F440C0182F76
:20062000893008F018E0811B8093600080916E0080FF02C003EC01C00BE48F5F80936E0034
:2006400020919F003091A00086FD05C0912FF901A7E8B0E00DC0912FF901A7E8B0E003C05F
:2006600084918D9331969150D8F704C081918D939150E0F7C901810F911D9093A000809342
:200680009F00612F87E890E08DD2183019F08FEF80936000009386001C5F109361009AE099
:2006A00080B3857061F49150D9F71092A20010929C0005C090E084CF90E020EC82CFDF91C5
:2006C000CF911F910F9108951F93DC01162F8091620084FF07C08091910098E88927809357
:2006E000910003C08AE580936200912FE2E9F0E002C08D9181939150E0F7612F82E990E050
:2007000051D21C5F109362001F9108951F920F920FB60F9211248F9380917300823028F08C
:20072000809173008150809373008F910F900FBE0F901F901895FC018DE790E09093A000B3
:2007400080939F0080818076803291F58181813019F488E090E00895893051F48681978166
:20076000019731F581E0809379008FEF90E00895823019F485E890E014C08A3021F4838100
:200780008093850007C0833041F48381882381F410926A0080E090E008958B3049F48AE60D
:2007A00090E09093A00080939F0081E090E0089580E090E00895FC0180917900882329F02E
:2007C000613019F4808180936F001092790081E090E0089588E0EDE7F0E011928A95E9F7C1
:2007E00080917B00882339F08091780080937D0010927B0021C0E0916800F09169008491AA
:2008000080937A00982F991F9927991F990F90937D00982F9F7790937F00882331F03196FA
:20082000F0936900E093680004C0109269001092680081E080937B0081E090E0089520910A
:2008400071003091720099272115310541F0FC01EF77F070EE0FFF1FE20FF31F0BC0FC01EE
:20086000EF77F070EE0FFF1F8091660090916700E80FF91F25913491E22F10927200109247
:200880007100253608F450C0233760F120917400E337F1F0FF27EE0FFF1FEF51F0408591EE
:2008A000949190936900809368008091750028232093740080917700882309F061C081ED59
:2008C00090E090936700809366001092760029C081ED91E090937200809371002260209377
:2008E00074001FC02D36A0F0ED568E2F817080937700E695E0937600FF27EE0FFF1FE85E4C
:20090000FB4F85919491909367008093660009C0FF27E459FC4FE491809174008E2B809312
:20092000740080E090E00895222351F188E0EDE7F0E011928A95E9F720937F00832F9927FD
:20094000882311F48091740080937D0080917D0080937800809174009091750089238093DF
:20096000740080917700882341F481ED90E090936700809366001092760081E090E0089534
:2009800080E090E008951F93182F662359F080917C00882309F45FC080916C0080954FDF0B
:2009A000282F5AC060916C00462F5527282F3327C9018095909584239523892B59F081E006
:2009C00080937C00612360936C00809163008093700041C04095509524233523232BD9F13C
:2009E00080916500882331F080917C00882329F081E003C01F3F99F402C0882381F0809166
:200A00007000813011F420E004C0862F809517DF282F10936C0010927C00222339F4809125
:200A20007000813011F020E00DC020E08091680090916900892B31F48EE194E0909369007C
:200A4000809368001092700080916500882321F010936C0001C020E0822F99271F91089549
:200A60001F9386B310B3107C8F73182B90916B009117B1F080917300882329F48091640061
:200A80008093730019C0809173008130A9F460E0812F79DF982F10936B00109273000DC026
:200AA00080917000823041F461E0892F6CDF982F81E08093700001C090E0892F99271F9186
:200AC0000895CFE5D4E0DEBFCDBF88E190E02FE00FB6F894A89581BD0FBE21BD8FE388BBD4
:200AE00017BA88E385BB97E094BB8AEF82BB91BB8CE28A95F1F782E081BB85E083BF8FE287
:200B000083BD8EE085BD89B7806889BFA4DC789410E000E0CDE7D0E0A895A7DC112351F47C
:200B20008091680090916900892B11F053DE01C097DF182F08B600FE15C081E088BF809104
:200B40007000833028F08091700081508093700080918500882331F0053018F4082F11E0BA
:200B600003C005501123C1F28091620084FFD4CF68E0CE01A9DD10E0CFCFA82FB92F80E093
:200B800090E041E050EA60956F5F58F42D9138EF82279795879510F0842795273F5FC8F3E5
:200BA000F3CF0895EADF8D939D930895CF93CFB7CF93809BFECF809B09C0809B07C0809B0D
:200BC00005C0809B03C0809B01C0A3C0DF93C0919E00DD27CB55DF4F809B02C0DF91EBCF79
:200BE0002F930F931F9300B32FEF00FB20F94F933F9310B34FEF012700FB21F93BE031C0FC
:200C00004E7F012F10B3216028C0102F4D7F2260000000B329C04B7F2460012F000010B341
:200C20002BC010B3477F28602AC04F7E00B320612CC04F7D10B320622FC04F7B00B32064E0
:200C400032C0422700B349934FEF0000102710FB20F910B31570C9F1297F91F2012700FBC1
:200C600021F900B3237F89F2315058F1102710FB22F910B3277E79F2012700FB23F92F7CA6
:200C800081F200B3102710FB24F92F7971F200C010B3012700FB25F92F7359F200C000B3A0
:200CA000102710FB26F9223040F200C010B3012700FB27F9243028F64F77206810B3000006
:200CC000F9CF10E41ABF002719C03B503195C31BD04010E41ABF0881033CF9F00B34E9F0AA
:200CE00020919C001981110F1213EDCF4A81441F093641F10D3211F0013E29F70093A30098
:200D00003F914F911F910F912F91DF91CAB7C6FD50CFCF91CFBFCF9118950091A3000023EE
:200D200079F31091A1001123A1F53430A2F13093A10000939D0010919E003BE0311B309347
:200D40009E0029C00091A10001301CF50AE54F7049F43091610034FD20C000936100C6E8D8
:200D6000D0E01FC03091620034FD17C000936200C1E9D0E016C0052710E002BB1FC00527B0
:200D800022C0052727C005272CC0052710E002BB33C04AE503C042ED01C0432FC4E1D0E0D1
:200DA00032E011B31560909A02B311BB5F9355E020E820FF052702BB279517951C3FD8F675
:200DC00020FF0527279502BB17951C3FC0F620FF05272795179502BB1C3F98F620FF0527EE
:200DE000279517951C3F02BB70F600C0499120FF052702BB279517951C3F38F620FF05272F
:200E0000279502BB17951C3F38F520FF05272795179502BB1C3F10F520FF052727951795A2
:200E20001C3F02BBE8F4242F3A9519F60A7F5F9102BB1091A200110FC651D04011F0109329
:200E40009C0010E41ABF016011B31A7F402F4A7F02BB11BB42BB54CF0527D3CF0527D8CFE9
:200E60000527DDCFA1E1B0E0E7E3F7E004C41C01798B688B5A01FC0117821682838181FD00
:200E800003C08FEF9FEF5BC1882445C1282D332720FF2EC1892D80538A3008F437C1F7E6E4
:200EA000F91554F185E698160CF04DC093E5991609F461C09915ACF0EBE29E1609F426C1C9
:200EC000E9154CF0F0E29F1609F420C123E2921609F006C11BC1892D8D52823008F000C12A
:200EE00015C183E6981699F189150CF44FC098E5991609F0F5C021C0E0E79E16D1F0E915D9
:200F000064F0FCE69F16E1F08FE6981609F462C099E6991609F0E4C039C0E5E79E1609F492
:200F20005BC0F8E79F1649F023E7921609F0D8C013C038E7932E80E14EC090E19F874CC0C1
:200F4000E4E08E2AE3C09FE3C92EC501F6C0C5010296F501C080F1C0F501C080D180F601BA
:200F600001900020E9F73197EC19EF8722E030E0A20EB31E82C085010E5F1F4FF501C08031
:200F8000D180C601A2D28F8758018DC022FF08C0F50180819181A281B38124E030E009C0E3
:200FA000F50180819181AA2797FDA095BA2F22E030E0A20EB31E6C017D01B7FF22C032E07D
:200FC000832AF094E094D094C094C11CD11CE11CF11C17C088E08F8722FF08C0F5018081AB
:200FE0009181A281B38124E030E007C0F50180819181AA27BB2722E030E0A20EB31E6C01F1
:201000007D0187017601CE0101969E878D879F85492E552466247724C801B701A3019201C3
:2010200008D36A301CF0690D615201C0605DED85FE856193FE87ED87C801B701A3019201EE
:20104000F8D279018A01211531054105510521F7CC24DD24760181FE04C0B1018DE290E065
:2010600080D2F3E69F1631F4B1018C2D992787FD90953BC023E7921681F4860108C0F8012D
:2010800081918F01B101992787FD90956AD2FF85F150FF87FF3F99F729C023E5921619F09C
:2010A0000D851E8517C0860107C0F8018491B101992757D20F5F1F4FFF85F150FF87FF3FC8
:2010C000A1F714C0F80182918F01B101992787FD909547D2CE0101960817190799F706C0D9
:2010E000B101892D992787FD90953BD288240EC0F5E29F1629F42AE02F8781E0882E06C052
:20110000B101892D992787FD90952BD2888999890196998B888BF101838183FF04C0E88953
:20112000F989949003C0E889F9899080992009F0ADCEF1018681978102C05C0195CFE2E1BF
:201140006196B5C2A9E0B0E0E7EAF8E094C22C01798768874A01FC0117821682838180FDF3
:2011600005C02FEF3FEF3C832B83AAC11E821D828FEF9FEF9C838B83662477241A821982B2
:20118000222472C120FE5EC1853219F49EEF292265C1992787FD9095B4D2382EACE68A174F
:2011A00069F1A817A4F0B4E68B1709F46EC0B8172CF0E3E68E1709F02BC123C0F8E68F1776
:2011C00009F44CC129E6821709F022C15EC033E7831749F138174CF08FE6381609F44CC01E
:2011E00090E7391609F014C14CC0A5E78A1709F44AC0B8E78B1709F00BC143C0E4E02E2AF6
:201200002DC1D4010D911C91C20168D13C01BFEF8F3F9B0709F438C1E2E0F0E08E0E9F1E88
:20122000D8018D93F5C084010E5F1F4FF401E080F180C20153D13C0155D2892BD1F7FFEF25
:201240006F16FFEF7F0651F41FC1C3014BD2892B29F05701B201C301B1D10AC0D7016D92D1
:201260007D01C2013BD13C018F5F9F4F71F75701F50110824801CCC0E2E02E2AF8E0FF8377
:2012800004C020E12F8332E0232AC20127D13C0129D2892BD1F78FEF68168FEF780609F414
:2012A000F1C0862D8D3219F08B3251F402C098E0292AC20113D13C018F5F9F4F09F4E2C014
:2012C000B0E36B1671F5AA24BB246501C20106D13C01EFEF8F3F9E0709F46DC012D288378C
:2012E000D9F4FFE63F1631F024E6321619F035E7331621F4B201C30161D15DC0C201EED0AA
:201300003C018FEF68168FEF780619F490E19F8352C0A0E1AF8305C0B9E63B1611F4E8E0B1
:20132000EF83EE24FF248701C301EBD120EDC22E2FEFD22EC80ED91EFAE0CF16D1043CF056
:20134000C601C19762F029ED3FEFC20ED31ED7FC06C03F81832F9927C816D90634F0570113
:201360006801B201C3012AD11DC08F81282F332744275527C801B7013DD17B018C01C601AE
:20138000AA2797FDA095BA2FE80EF91E0A1F1B1FC201A4D03C019FEF69169FEF790621F6B5
:2013A0005701680123FE07C0AA24BB246501AE18BF08C00AD10A222D3327C90186709070D6
:2013C000069741F4D401ED91FC91A082B182C282D38207C021FF0AC0D401ED91FC91B182A9
:2013E000A082E2E0F0E08E0E9F1E12C0C401029622FF08C0D401ED91FC91A082B182C2824F
:20140000D38205C0D401ED91FC91B182A0824C01F2018681978129813A812817390744F402
:201420008D819E8101969E838D831C821B8208C09EE6391639F5AFEF6A16AFEF7A0611F175
:2014400022240CC0853251F4F2010680F781E02DFA83E983FAE0FF8381E0282E2885398519
:201460002F5F3F4F39872887F201838183FF04C0E885F985849103C0A885B9858C918823AE
:2014800009F080CE20FE0FC0F2018681978129813A81281739073CF48D819E8101969E830D
:2014A0008D831C821B829FEF69169FEF790621F4AD81BE81AB2B21F0ED81FE81FC83EB8384
:2014C0008B819C81E2E12996F2C0FC0105900020E9F7809590958E0F9F1F0895CF93DF9317
:2014E000EC012B81822F992780FF15C086FF0AC02F7B2B838E819F8101969F838E838A81E3
:2015000099272CC082FF12C0E881F9818081882329F420622B838FEF9FEF20C0282F332753
:2015200027FD30953196F983E88311C0EA85FB85CE0109959C0197FF0AC08B812F5F3F4FC2
:2015400011F490E101C090E2892B8B83E4CF8E819F8101969F838E83822F9927DF91CF9133
:2015600008950F931F93CF93DF938C01EB018B81992781FF1BC082FF0DC02E813F818C813C
:201580009D812817390764F4E881F9810193F983E88306C0E885F985802F0995892B31F421
:2015A0008E819F8101969F838E8302C00FEF1FEFC801DF91CF911F910F910895AC01FB0135
:2015C0002381822F992780FF12C086FD10C08FEF4F3F580761F0428320642F7D23838681F4
:2015E0009781019797838683842F992708958FEF9FEF0895629FD001739FF001829FE00D7C
:20160000F11D649FE00DF11D929FF00D839FF00D749FF00D659FF00D9927729FB00DE11DD4
:20162000F91F639FB00DE11DF91FBD01CF0111240895A1E21A2EAA1BBB1BFD010DC0AA1F63
:20164000BB1FEE1FFF1FA217B307E407F50720F0A21BB30BE40BF50B661F771F881F991F37
:201660001A9469F760957095809590959B01AC01BD01CF0108952F923F924F925F926F924F
:201680007F928F929F92AF92BF92CF92DF92EF92FF920F931F93CF93DF93CDB7DEB7CA1B4B
:2016A000DB0B0FB6F894DEBF0FBECDBF09942A88398848885F846E847D848C849B84AA84EA
:2016C000B984C884DF80EE80FD800C811B81AA81B981CE0FD11D0FB6F894DEBF0FBECDBF97
:2016E000ED010895911113C0803251F08A3041F08C3031F08D3021F0893011F08B3099F75C
:2017000008958F9309D08F9109F08062089599278827089585FDFBCF80629111F8CF81363F
:20172000ECF38B37DCF70895FF5A5A190A01D1001E0401FFFF00FFFFFFFFFFFFFFFFFFFFD9
:20174000FFFFFFFFFFFFFFFFFFFFFFFFFFFFFFFFFFFFFFFFFFFFFFFFFFFFFFFFFFFFFFFFA9
:20176000FFFFFFFFFFFFFFFFFFFFFFFFFFFFFFFFFFFFFFFFFFFFFFFFFFFFFFFFFFFFFFFF89
:20178000FFFFFFFFFFFFFFFFFFFFFFFFFFFFFFFFFFFFFFFFFFFFFFFFFFFFFFFFFFFFFFFF69
:2017A000FFFFFFFFFFFFFFFFFFFFFFFFFFFFFFFFFFFFFFFFFFFFFFFFFFFFFFFFFFFFFFFF49
:2017C000FFFFFFFFFFFFFFFFFFFFFFFFFFFFFFFFFFFFFFFFFFFFFFFFFFFFFFFFFFFFFFFF29
:2017E000FFFFFFFFFFFFFFFFFFFFFFFFFFFFFFFFFFFFFFFFFFFFFFFFFFFFFFFFFFFFFFFF09
:201800003FC06AC158C057C056C055C054C053C052C051C050C04FC04EC04DC04CC04BC0A9
:201820004AC049C048C012010101FF000008C016DC05000101020001090212000101008016
:201840000A090400000000000000040309041C037700770077002E00660069007300630006
:2018600068006C002E0064006500160341005600520055005300420042006F006F0074001D
:2018800011241FBECFE5D4E0DEBFCDBF10E0A0E6B0E0EEEAFFE102C005900D92A436B1075F
:2018A000D9F710E0A4E6B0E001C01D92A03AB107E1F765D37BC3A4CF84E690E08093970007
:2018C0000B968093960085B7836085BF8BB780648BBF08950F931F93CF93DF9360919C0099
:2018E000662309F493C0635067FD8EC080919600282F2F5FE901809199008D3209F068C0AA
:20190000683009F07BC08881807609F057C0109294008981882321F41092950022E03FC0B4
:20192000853021F48A8180939D0038C0863029F58B81813019F486E298E104C0823021F420
:2019400088E398E122E117C0833079F48A81882321F48AE498E124E00EC0813021F48EE4ED
:2019600098E12CE108C0823019F020E030EC18C08AE698E126E130EC15C0883029F421E0B3
:2019800030E88FE990E00EC0893021F48A8180939F0004C08A3011F421E001C020E030E891
:2019A00084E990E090939B0080939A008F81882339F58E81821720F5282F22C0CE0144D21B
:2019C000282F8F3FE1F488818823B4F42E8114C080917A0087FD12C0CE0172D28F3F39F43F
:2019E0008EE180938B0082E08093610004C0882311F020E001C02FEF30E002C020E030E8CB
:201A000030937A002093600010929C00909160009F3F09F445C08091610087FF41C0692F46
:201A2000993008F068E0961B9093600080917A0080FF02C003EC01C00BE48F5F80937A0083
:201A400020919A0030919B0086FD05C0962FF901ACE8B0E00DC0962FF901ACE8B0E003C041
:201A600084918D9331969150D8F704C081918D939150E0F7C901860F911D90939B0080932E
:201A80009A007727162F8CE890E0CCD1183018F48FEF8093600000938B001C5F1093610066
:201AA00080B3857019F010927B0011C080917B00882369F494E680B3857049F49150D9F7E3
:201AC00081E080937B0010929D0010929800DF91CF911F910F9108950F930FB70F93809BBC
:201AE000FECF809B06C0809B04C0809B02C0000000C01F933F932F9331E014E000B3102787
:201B000010FD32E0102F3A95C9F700FDE5C000B3102717952FE72795DF9310B301270795D5
:201B20002795CF93C091970000B31027179527953BE0D0E04F9310B30127079527954FEF1F
:201B4000000055C0809BFECF809B06C0809B04C0809B02C0000000C0DF9100C0CDCF10B39C
:201B6000157079F1407C2C6F13C000B3057049F141782C6F15C0057021F1102F2C6F00B3AD
:201B800019C000B30570E9F04E7F2C6F18C038F300B30570B1F0102717952795243028F329
:201BA00010B3012707952795422749934FEF00B3243008F3102717952795243010F310B3A4
:201BC0001570E1F10127079527952430F0F000B30570A1F11027179527952430E0F010B3BA
:201BE0000127079527953A9541F12430D0F000B3057021F11027179527952430C0F010B3B0
:201C00000127079527952430C2CF10B31570B1F04C7F2C6FDCCF00B3057081F0487F2C6F6A
:201C2000DECF10B3157051F0407F2C6FE0CF00B3057021F0407E2C6FE2CF3BC03C2FC0916B
:201C400097003C1B00E433300ABF98F108811981412F1F77209198000D3279F1013E69F149
:201C60000936C1F00777033421F510919E00112301F100919C000030C1F53430CAF130934F
:201C80009C001093990000919600C0939600009397002EC0121769F4309161003F3F29F104
:201CA0000FEF00936100CBE8D0E025C0002700939E004F91CF91DF910FC01217B9F70093A7
:201CC0009E000FEF00936000009361004F91CF910AB706FD37CFDF9100E40ABF2F913F91CA
:201CE0001F910F910FBF0F911895C3E6D0E002C0C2E6D0E032E05F9302B30A7F016002BBA6
:201D000055E011B3156011BB20E80FC0052710E002BB10C0052710E0089402BB13C0052795
:201D200010E015C0052710E019C020FF052702BB279517951C3F50F720FF0527279502BB13
:201D400017951C3F38F720FF05272795179502BB1C3F28F720FF0527279517951C3F02BB98
:201D600008F700C0499120FF052702BB279517951C3F80F520FF0527279502BB17951C3FBF
:201D800068F520FF05272795179502BB1C3F58F520FF0527279517951C3F02BB38F5242F83
:201DA0003A9519F60A7F5F9102BB32E03A95F1F710919D00C556D04011F010939800016040
:201DC00011B31A7F02BB0A7F4F91CF9111BB02BBDF9182CF052710E002BBCACF052710E048
:201DE000089402BBCDCF052710E0CFCF052710E0D3CFA82FB92F8FEF9FEF41E050EA61509F
:201E000070F02D9138E0722F782796958795269570FF02C0842795273A95A9F7F0CF80956F
:201E200090950895E6DF8D939D930895F89481E180935700E89581E08BBF1BBEE0917C00E8
:201E4000F0917D0009950895FC018181813011F4EDDF25C0823009F581E080937E0083813D
:201E600022819927582F44273327422B532B509388004093870010928A0010928900E19932
:201E8000FECFF89483E0FA0180935700E895789407B600FCFDCF2FEF0AC0833011F020E077
:201EA00006C010927F0080E48093800022E08FE790E090939B0080939A00822F99270895E3
:201EC000DF92EF92FF920F931F93CF93DF938C01E62E80917E00813019F08FEF90E047C078
:201EE00060918700709188004091890050918A00DB01A40FB51FC0E0D0E081E0F82EF5E00D
:201F0000DF2E2CC0F894F801E80FF11D2081818133279927982F8827282B392B0901FD014C
:201F2000F0925700E895112478944E5F5F4F229612964034510590F050938A00409389003C
:201F4000F894FB01D0925700E895789407B600FCFDCF10927E0081E090E009C08C2FCE15DA
:201F600088F250938A004093890080E090E0DF91CF911F910F91FF90EF90DF9008958FEF96
:201F800088BB17BA15BA14BA8AEF82BB82E081BB869903C086B3807309F048DF81E08BBF63
:121FA00082E08BBF89DC789495DCFECFFFCFFFFFD25ADC
:00000001FF
